:10000000D82AA500841780048413FA30B200B30103
:100010000722A60AAF0AAA01AB0100082505B20013
:10002000000000082505B300320633052506031934
:10003000AA0A0319AB0A3308B200AE030319AF03CF
:100040000319A60B10282A081D2A8030A100FE30B3
:100050005121013051217530A70030306229A101B2
:10006000A117B600B608031D372803013828013050
:10007000B6020310A20CA20CA20CC0302205403E16
:10008000B607FE30512136085129A101A117B6004B
:10009000FE30512136085129A01124080319A0155A
:1000A0000530A3002730AB00103062200330AB00D6
:1000B000E8306220AB0164306220AB010A3062207C
:1000C0002E086928AA002F08A7002E08A600EB21F9
:1000D0002608A600A3030319A011240803197328F6
:1000E000230203187A282608031DA011A0197A28D4
:1000F000303E51290800C900BA1F80282D305121F7
:10010000BC0F8728BB0F8728BA0A0319BA0AC10196
:10011000C201C301C401BA176A30B9070310BA0C8F
:10012000BB0CBC0CC40CC30CC20CC10CB90F8E2888
:100130003C083902BC07B9023B083A02BB07BA02C5
:10014000A401DA202E305121CA010310410DBC0058
:10015000420DBB00430DBA00440DB900CA0D031097
:10016000BC0DBB0DBA0DB90DCA0D4108BC07420844
:100170000318420FBB0743080318430FBA0744088C
:100180000318440FB9070318CA0F0310BC0DBB0DA9
:10019000BA0DB90DCA0D4A08303E51213C08C100C4
:1001A0003B08C2003A08C3003908C400C90BA428A0
:1001B00003101D2AA0112408031DE128A0150A30F0
:1001C000A4003C08A9003B08A8003A08A700390889
:1001D000A600A301B101B001AF010A30AE00712148
:1001E000A30A23082402031DEA282E08031DA011D8
:1001F000A01DFC28240BFF282E08303E5121A40B03
:10020000E1281D2AB30006118611831606118611F6
:100210000F30860583123308A0182C293E30A70022
:10022000803062213330B20040211330A700883083
:1002300062214021643061214021643061212230FB
:10024000B200402128302B210C302B2106302B21ED
:10025000A01433082C292014B200201C3A2986113E
:10026000033C031C3F293F210730A700D030622107
:10027000031408002014FE3C03194F298615201C86
:10028000201006150F3086053208F039860400006C
:100290000611B20E000020184029323061213308C7
:1002A0001D2AA11B02290800AB01AA00FF30AA07E2
:1002B000031CAB07031C1D2A0330A700E630622194
:1002C0005629A701FC3EA600A709031C6D29FF3093
:1002D0000000A60703186829A6070000A70F6729D2
:1002E0000800290831068039B300A91F8229A60910
:1002F000A709A809A909A60A0319A70A0319A80AA0
:100300000319A90AB11F8F29AE09AF09B009B109B4
:10031000AE0A0319AF0A0319B00A0319B10AAA01F8
:10032000AB01AC01AD01BD01BE01BF01C00131088F
:1003300030042F042E040319CD292030B2000310FD
:10034000A60DA70DA80DA90DBD0DBE0DBF0DC00DAD
:1003500031084002031DB62930083F02031DB629AB
:100360002F083E02031DB6292E083D02031CC72993
:100370002E08BD022F08031C2F0FBE023008031CDD
:10038000300FBF023108031C310FC0020314AA0D45
:10039000AB0DAC0DAD0DB20B9F29B31FDA29AA0925
:1003A000AB09AC09AD09AA0A0319AB0A0319AC0AD7
:1003B0000319AD0A3D08AE003E08AF003F08B0008B
:1003C0004008B1002A08A6002B08A7002C08A800A6
:1003D0002D08A9001D2AAF01AE011030B200270D73
:1003E000AE0DAF0D2A08AE022B08031C2B0FAF0277
:1003F0000318012A2A08AE072B0803182B0FAF0792
:100400000310A60DA70DB20BEF2926080800103027
:10041000B800A701A601B30CB20C031C152A2A08C8
:10042000A6072B0803182B0FA707A70CA60CAF0CC9
:10043000AE0CB80B0B2A2E0808008313831203138B
:1004400008004208BF004606CD004108003A031DDF
:100450004508003A0319732AC1077E30031C342A69
:10046000C1020318752A372AC102031C722A4408E4
:10047000BD004308BE00BF17C617C401C301C201B7
:100480001830CC00BF0CBE0CBD0C031C512A480810
:10049000C40747080318470FC30746080318460F49
:1004A000C207C20CC30CC40CCC0B422AC21B602A6C
:1004B000C40DC30DC20DC1080319722AC1033F0D3B
:1004C0004B1F712A031C712AC40F712AC30F712A92
:1004D000C20F712A0314C20CC30CC40CC10A031945
:1004E000752A7C2A4B15C101782ACB14FF30C10034
:1004F000C401C3018030C200CD1B7F2AC2131D2A54
:10050000C301C4019630CC00CD13C41F932AC40983
:10051000C309C209C109C10F922AC20F922AC30A94
:100520000319C40ACD17C4080319AE2A4B1FA52A04
:10053000C41FA52AC20FA52AC30FA52AC40FA52A26
:100540000314C40CC30CC20CCC0A0830CC074208FC
:10055000C1004308C2004408C300C32AC308031DE6
:10056000C32A0830CC024208031DBF2A0830CC023F
:100570004108031DBE2A4408CC00CD2AC101C30096
:100580004108C200C101C31BCB2A0310C10DC20D1B
:10059000C30DCC03C32ACD1FC3134108C4004C08AC
:1005A000C1004308CC004208C3004C08C2001D2A09
:1005B00083014030CB00A0014F308316850003300B
:1005C0008600073083129F00FE3002214030022156
:1005D0000E30022111300221103002211030022190
:1005E00010300221153002210E300221003002218C
:1005F000FE300221483002210A3002210E30022151
:10060000113002211130022111300221113002215A
:100610000E30022100300221FE3002215030022132
:100620000A30022111300221113002211130022141
:1006300011300221113002210E300221003002213E
:10064000FE30022158300221043002210E300221F6
:10065000043002210430022104300221043002213E
:100660000E30022100300221FE30022160300221D2
:100670000E30022111300221103002210E300221F1
:1006800001300221153002210E30022100300221FA
:10069000FE300221683002210E300221003002219A
:1006A0000F300221103002211730022111300221B7
:1006B0000F30022100300221FE30022100300221E1
:1006C00000300221003002210930022109300221CC
:1006D000093002210E3002210830022164305421F9
:1006E0002520CF01CE01D101D001D501D401D30104
:1006F000D201D901D801D701D601DA01DC01DE012E
:10070000DD01DB012C240730AB00D0305521252042
:100710008030A100C03045204330022150300221FA
:1007200053300221C5304520433002215030022190
:100730004D300221CA3045200630022153300221BB
:10074000763002212F300221683002210330AB00C5
:10075000E830AA000530840002300120CE002B08CA
:10076000CF008030A100CF3045202A3002218030D8
:10077000A1004520A4014F08AF004E08AE004C2058
:10078000DC0A4E08D0074F080318013ED1073B3062
:100790005C02031DCC2BD523323054218030A100C4
:1007A000CF30452020300221882B8030A100452009
:1007B00020300221022102210221022102210221F4
:1007C0000221022102210221022102210221022111
:1007D00002218030A1004520A4014F08AF004E083F
:1007E000AE004C208030A10085304520A401510886
:1007F000AF005008AE004C205008C1005108C200A4
:1008000080221130C800C730C7003A30C6007730A8
:10081000C50021224408D5004308D4004208D30073
:100820004108D2008030A1008A3045205508BC0024
:100830005408BB005308BA005208B90002307B20AC
:10084000DC01D101D001D501D401D301D201CF0106
:10085000CE013230542108001030DB0002305B0240
:10086000031C482C8030A1000130A2005B0831201D
:100870002A3002218030A1000130A2005B0A312021
:10088000203002212D3054210130DB0203182E2CA0
:100890001030DB0004305B02031C642C8030A100AC
:1008A0000130A2005B083120543002218030A100C9
:1008B0000130A2005B0A3120203002212D3054216A
:1008C0000130DB0203184A2C1030DB0006305B02DB
:1008D000031C802C8030A1000130A2005B08312075
:1008E000413002218030A1000130A2005B0A31209A
:1008F000203002212D3054210130DB020318662CF8
:100900001030DB0008305B02031C9C2C8030A100FF
:100910000130A2005B083120323002218030A1007A
:100920000130A2005B0A3120203002212D305421F9
:100930000130DB020318822C1030DB000A305B022E
:10094000031CB82C8030A1000130A2005B083120CC
:10095000453002218030A1000130A2005B0A312025
:10096000203002212D3054210130DB0203189E2C4F
:100970001030DB000C305B02031CD42C8030A10053
:100980000130A2005B083120493002218030A100F3
:100990000130A2005B0A3120203002212D30542189
:1009A0000130DB020318BA2C1030DB000E305B0282
:1009B000031CF02C8030A1000130A2005B08312024
:1009C0002A3002218030A1000130A2005B0A3120D0
:1009D000203002212D3054210130DB020318D62CA7
:1009E0008030A1008E3045202030022102210330CA
:1009F000AB00203055218030A100C030452052305E
:100A0000022141300221443002215930022141307B
:100A1000022153300221593002214F3002214E3041
:100A2000022120300221013002214C30022100300D
:100A3000022102300221433002210230022107301C
:0A0A4000AB00D03055210800242D32
:02400E00223F4F
:00000001FF
